:103800000C942A1C0C94451C0C94451C0C94451CCF
:103810000C94451C0C94451C0C94451C0C94451CA4
:103820000C94451C0C94451C0C94451C0C94451C94
:103830000C94451C0C94451C0C94451C0C94451C84
:103840000C94451C0C94451C0C94451C0C94451C74
:103850000C94451C11241FBECFE5D4E0DEBFCDBFC4
:1038600010E0A0E6B0E0E4ECFCE302C005900D92AD
:10387000A036B107D9F710E0A0E6B0E001C01D9274
:10388000A336B107E1F70C945D1C0C94001C81E495
:103890000E94391E86E50E94391E82E50E94391E6B
:1038A00082E40E94391E8FE40E94391E8FE40E9438
:1038B000391E84E50E94391E0895CFE5D4E0DEBFAD
:1038C000CDBFC0E0D0E001E08FEF8BBB60E08BE0CC
:1038D00090E00E942F1E05BF82E085BFCF9B06C0EF
:1038E00081E085BF15BEFE0109950FC00E944E1EE6
:1038F0008B3141F40E944E1E8335E1F70E94471C34
:1039000000E003C08FE30E94391E002339F70E94B4
:103910004E1E682F813611F489E5B7C08134A9F4B1
:103920000E944E1E99279093610080936000182F8B
:1039300000270E944E1E9927082B192B000F111FDC
:1039400010936100009360005CC0823641F489E509
:103950000E94391E80E00E94391E80E896C08234A1
:1039600089F40E944E1E9927182F00270E944E1E90
:103970009927082B192B0E944E1E682FC8010E9400
:10398000481D83C0873689F40E944E1E9927182F40
:1039900000270E944E1E9927082B192B0E944E1EAD
:1039A000682FC8010E94C31DB2CF853661F5809192
:1039B00062008537F9F4109261001092600063E0B4
:1039C00080916000909161000E94FE1D61E18091F4
:1039D0006000909161000E94FE1D809160009091B6
:1039E000610080589F4F90936100809360008050E9
:1039F000984328F361E180916000909161000E94FA
:103A0000FE1D8DE042C0853451F488E190E028E04D
:103A10000FB6F894A89581BD0FBE21BDF2CF8035B9
:103A200081F38C3471F3803711F483E52EC0843731
:103A300029F485E70E94391E80E027C0885782302C
:103A400018F40E944E1EDDCF643529F40E944E1EEC
:103A500080936200D6CF633519F40E94471C57CF7C
:103A6000663529F480E30E94391E82E30EC0633775
:103A700041F483E00E94391E84E90E94391E8EE1E0
:103A800004C06B3109F443CF8FE30E94391E3FCF4E
:103A9000DF92EF92FF920F931F93CF93DF937C01FE
:103AA000D62EC0916000D091610080916200853770
:103AB00009F05FC086E46817D1F50E944E1E082FFA
:103AC00011270E944E1E9927982F8827082B192B03
:103AD0006091600070916100C8010E940D1E80918C
:103AE0006000909161000296909361008093600065
:103AF0008EEF9FEFE80EF91EE114F104F1F6C078A5
:103B000065E0CE010E94FE1D61E1CE010E94FE1D16
:103B100080916000909161009C012078821793074A
:103B200031F020583F4F309361002093600095E4BE
:103B3000D916E1F4809160008EBB80916000909175
:103B40006100292F33272FBB01969093610080934A
:103B500060000E944E1E8DBBE29AE19AE199FECF71
:103B60000894E108F108E114F10421F78DE090E0F8
:103B700002C080E090E0DF91CF911F910F91FF9004
:103B8000EF90DF9008950F931F93CF93DF93EC0195
:103B90006534B1F4809160008EBB8091600090919B
:103BA0006100292F33272FBB0196909361008093EA
:103BB0006000E09A8DB30E94391E219759F719C011
:103BC00060E080916000909161000E94201E8C0155
:103BD0000E94391E812F99270E94391E8091600012
:103BE000909161000296909361008093600022970B
:103BF00039F7DF91CF911F910F91089507B600FC1F
:103C0000FDCFE199FECFFC0160935700E895FFFFDF
:103C1000000007B600FCFDCF08959C0107B600FC2C
:103C2000FDCFE199FECF81E00901FB0180935700B0
:103C3000E895FFFF0000112407B600FCFDCF0895B2
:103C400007B600FCFDCFE199FECFFC0160FD60935B
:103C50005700C895802DE395C895902D08959C0137
:103C6000832F992780BD29B988E18AB986E880BD6C
:103C7000089520E030E08CB90FB607FE0BC05E99C6
:103C80000BC02F5F3F4F5E9907C087E22031380796
:103C9000C4F302C05E9BFECF5E9A089580E090E080
:103CA0000FB607FE0AC05F990AC001965F9907C068
:103CB00027E280319207CCF302C05F9BFECF8CB12C
:043CC00099270895A3
:0400000300003800C1
:00000001FF
